:1000740093070000638807003725000013050599DE
:100084006F10901667800000972100009381C17A59
:10009400138541C3138681C53306A640930500002A
:1000A400EF10006F17250000130545946308050041
:1000B400172500001305C58DEF101013EF10806392
:1000C400032501009305410013060000EF0050537F
:1000D4006F10405F130101FF2324810083C7C1C354
:1000E400232611006392070293070000638A070026
:1000F400372500001305050097000000E700000005
:1001040093071000238EF1C28320C10003248100D1
:10011400130101016780000093070000638C07004E
:1001240037250000938501C413050500170300005B
:100134006700000067800000130101FF232681008F
:100144001304010183A7C1C29387870003A7070093
:1001540023AAE1C283A741C393F7170093B71700FB
:1001640093F7F70F138507000324C100130101015E
:1001740067800000130101FF23268100130401019D
:1001840083A7C1C29387870003A7070023AAE1C2FC
:1001940003A741C3B7070100B377F70093B717006C
:1001A40093F7F70F138507000324C100130101011E
:1001B40067800000130101FE232E81001304010255
:1001C4002326A4FE83A7C1C29387870003A7070041
:1001D40023AAE1C283A741C393F71700639E0700D4
:1001E40083A7C1C2938747000327C4FE23A0E70067
:1001F400930700006F0080009307F0FF138507004A
:100204000324C1011301010267800000130101FFEF
:10021400232681001304010183A7C1C293878700A9
:1002240003A7070023AAE1C203A741C3B70701003C
:10023400B377F7006398070083A7C1C283A70700B9
:100244006F0080009307F0FF138507000324C100AB
:100254001301010167800000130101FE232E110028
:10026400232C8100130401022326A4FE6F00000343
:10027400130000008327C4FE83C70700138507000B
:10028400EFF05FF3130705009307F0FFE304F7FEB5
:100294008327C4FE938717002326F4FE8327C4FE16
:1002A40083C70700E39607FC930700001385070044
:1002B4008320C1010324810113010102678000002E
:1002C400130101FD232611022324810213040103D7
:1002D400232EA4FC232CB4FC232604FE032784FD34
:1002E4009307100063C6E700930700006F008009BE
:1002F400EFF0DFF12324A4FE032784FE9307F0FF2D
:10030400E308F7FE8327C4FE138717002326E4FEC1
:10031400138707008327C4FDB387E700032784FE00
:100324001377F70F2380E70013000000032584FEF2
:10033400EFF05FE8130705009307F0FFE308F7FE0B
:10034400832784FD9387F7FF0327C4FE6350F702D6
:10035400032784FE9307A000630CF700032784FEA1
:100364009307D0006306F7006FF09FF813000000B6
:100374008327C4FE0327C4FDB307F70023800700C7
:100384008327C4FE138507008320C102032481024E
:100394001301010367800000130101FC232E810275
:1003A400130401042326A4FC2324B4FC232404FE04
:1003B400232204FE832784FC63DE0704832784FC52
:1003C400B307F0402324F4FC232204FE6F008004CE
:1003D400032784FC9307A000B367F70213F7F70F12
:1003E400832784FE938617002324D4FE9386070074
:1003F4008327C4FCB387D700130707031377F70FCA
:100404002380E700032784FC9307A000B347F70287
:100414002324F4FC832784FCE34CF0FA832744FE72
:1004240063820702832784FE138717002324E4FED4
:10043400138707008327C4FCB387E7001307D002A0
:100444002380E700232604FE6F00C006832784FE72
:100454001387F7FF8327C4FEB307F7402320F4FE76
:100464008327C4FE0327C4FCB307F70083C7070030
:10047400A30FF4FC832704FE0327C4FC3307F7000F
:100484008327C4FE8326C4FCB387F6000347070012
:100494002380E700832704FE0327C4FCB307F70087
:1004A4000347F4FD2380E7008327C4FE93871700E6
:1004B4002326F4FE832784FE13D7F701B307F7003E
:1004C40093D71740138707008327C4FEE3C0E7F8D8
:1004D400832784FE0327C4FCB307F70023800700A7
:1004E400832784FE138507000324C1031301010439
:1004F40067800000130101FB232681041304010516
:100504002326A4FC2320B4FC2322C4FC2324D4FCEF
:1005140093070700A30FF4FA232404FE6F000009D5
:10052400832704FC93F7F700232EF4FC0327C4FD70
:100534009307900063C4E7028327C4FD13F7F70F02
:10054400832784FE8326C4FCB387F60013070703BE
:100554001377F70F2380E7006F0040028327C4FD61
:1005640013F7F70F832784FE8326C4FCB387F600B2
:10057400130777051377F70F2380E700832744FCDD
:100584009397C701032704FC1358470033E8070176
:10059400832744FC93D84700232004FD232214FD21
:1005A400832784FE938717002324F4FE832704FC07
:1005B400032744FCB3E7E700E39407F66F00400227
:1005C400832784FE138717002324E4FE1387070080
:1005D4008327C4FCB387E7000347F4FB2380E700C9
:1005E400032784FE832784FCE34CF7FC232604FEC4
:1005F4006F00C006832784FE1387F7FF8327C4FE9A
:10060400B307F7402322F4FE8327C4FE0327C4FC68
:10061400B307F70083C70700A301F4FE832744FE52
:100624000327C4FC3307F7008327C4FE8326C4FCD6
:10063400B387F600034707002380E700832744FEBF
:100644000327C4FCB307F700034734FE2380E70005
:100654008327C4FE938717002326F4FE832784FE92
:1006640013D7F701B307F70093D717401387070091
:100674008327C4FEE3C0E7F8832784FE0327C4FC72
:10068400B307F70023800700832784FE1385070040
:100694000324C1041301010567800000130101FD57
:1006A4002326810213040103232EA4FC232CB4FC6F
:1006B400232604FE232404FE930710002322F4FEC1
:1006C4006F00C0088327C4FD83C707002320F4FEFE
:1006D400032704FE9307F00263D2E704032704FE12
:1006E4009307900363CCE702032784FE9307070074
:1006F40093972700B387E7009397170013870700A2
:10070400832704FEB307F700938707FD2324F4FE31
:10071400930710002326F4FE6F0080028327C4FE93
:10072400639E0702032704FE9307D002631AF700AF
:100734009307F0FF2322F4FE930710002326F4FE10
:100744008327C4FD93871700232EF4FC8327C4FD5D
:1007540083C70700E39807F66F00800013000000CA
:10076400032784FE832744FEB307F7022324F4FE01
:10077400832784FD63880700832784FD0327C4FD42
:1007840023A0E700832784FE138507000324C10206
:100794001301010367800000130101FD2326810278
:1007A40013040103232EA4FC232CB4FC232604FEEF
:1007B400232404FE6F00000E8327C4FD83C70700B3
:1007C4002322F4FE032744FE9307F00263DAE702D0
:1007D400032744FE9307900363C4E70293071000C2
:1007E4002326F4FE832784FE13974700832744FEC1
:1007F400B307F700938707FD2324F4FE6F00C008B6
:10080400032744FE9307000663DAE702032744FE46
:100814009307600663C4E702930710002326F4FEDF
:10082400832784FE13974700832744FEB307F7000A
:10083400938797FA2324F4FE6F000005032744FEF0
:100844009307000463DAE702032744FE9307600476
:1008540063C4E702930710002326F4FE832784FE73
:1008640013974700832744FEB307F700938797FC49
:100874002324F4FE6F0040018327C4FE639407021F
:10088400930710002326F4FE8327C4FD93871700E3
:10089400232EF4FC8327C4FD83C70700E39E07F0DF
:1008A4006F00800013000000832784FD6388070025
:1008B400832784FD0327C4FD23A0E700832784FE48
:1008C400138507000324C10213010103678000009C
:1008D400130101FD2326810213040103232EA4FC2A
:1008E400232CB4FC8327C4FD2326F4FE6F000001EF
:1008F4008327C4FD93871700232EF4FC8327C4FDAC
:1009040083C70700E39607FE6F004002032784FDB8
:1009140093071700232CF4FC8327C4FD9386170048
:10092400232ED4FC034707002380E700832784FD9C
:1009340083C70700E39C07FC8327C4FD23800700CB
:100944000327C4FD8327C4FEB307F74013850700BC
:100954000324C1021301010367800000130101FD98
:100964002326810213040103232EA4FC232CB4FCAC
:10097400232AC4FC232604FE6F0000058327C4FD3C
:1009840013871700232EE4FC03C70700832784FD85
:1009940093861700232CD4FC83C707006306F70053
:1009A400930710006F0000048327C4FE9387170089
:1009B4002326F4FE0327C4FE832744FD6346F70081
:1009C400930700006F0000028327C4FD83C707005C
:1009D40063880700832784FD83C70700E39007FA31
:1009E40093070000138507000324C10213010103C8
:1009F40067800000130101FE232E8100130401020D
:100A04002326A4FEB7E7F505138707108327C4FE42
:100A14003347F70283A7C1C29387070123A0E700E6
:100A240093070000138507000324C1011301010289
:100A340067800000130101EC232E1112232C811274
:100A4400232A21132328311323264113232451134A
:100A54001304011483A781C393F707FF232AF4FC2B
:100A6400232C04FC6F00801F832744FD1389070097
:100A7400930900009307C4EC130700039306800056
:100A8400930509001386090013850700EFF09FA65C
:100A94001307C4ECB7270000938507AD13050700BF
:100AA400EFF01FE3232E04FC6F00000C832744FDAA
:100AB4002326F4FC0327C4FD832744FD3307F700F2
:100AC40083A781C3637EF7001307C4ECB727000034
:100AD400938547AD13050700EFF09FDF6F00000615
:100AE4008327C4FD0327C4FCB307F70083C70700AB
:100AF400138A0700930A0000930744EC13070003CA
:100B04009306200093050A0013860A001385070044
:100B1400EFF05F9E130744ECB7270000938587AD81
:100B240013050700EFF0DFDA130744EC9307C4EC76
:100B34009305070013850700EFF09FD90327C4FD31
:100B440093077000631CF7001307C4ECB727000079
:100B54009385C7AD13050700EFF09FD78327C4FD26
:100B640093871700232EF4FC0327C4FD9307F0009A
:100B7400E3DEE7F21307C4ECB7270000938507AE62
:100B840013050700EFF0DFD4232E04FC6F000008E8
:100B9400832744FD2328F4FC8327C4FD032704FD95
:100BA400B307F70003C707009307F00163FAE702EE
:100BB4008327C4FD032704FDB307F70003C7070019
:100BC4009307E00763EEE7008327C4FD032704FDD2
:100BD400B307F70083C707002300F4EC6F00C000DD
:100BE4009307E0022300F4ECA30004EC130704ECE5
:100BF4009307C4EC9305070013850700EFF05FCD5E
:100C04008327C4FD93871700232EF4FC0327C4FD18
:100C14009307F000E3DEE7F61307C4ECB727000000
:100C2400938547AE13050700EFF09FCA9307C4EC02
:100C340013850700EFF04FE2832744FD93870701F4
:100C4400232AF4FC832744FD93F7F70F63800702FC
:100C5400832784FD93871700232CF4FC032784FD4A
:100C64009307F000E3D2E7E06F0080001300000078
:100C7400B7270000138587AEEFF00FDE032744FD8E
:100C840023ACE1C2130000008320C11303248113A9
:100C94000329411383290113032AC112832A8112D0
:100CA4001301011467800000130101FE232E81004B
:100CB40013040102F36500C02326B4FEF36500C8E3
:100CC4002324B4FE832584FE2320B4FE232204FEC1
:100CD400832504FE9398050013080000232004FFD5
:100CE400232214FF8325C4FE138705009307000005
:100CF400832504FE33E6E500832544FEB3E6F500D0
:100D04002320C4FE2322D4FE032704FE832744FEAB
:100D140013050700938507000324C1011301010291
:100D240067800000130101FE232E810013040102D9
:100D3400F36520C02326B4FEF36520C82324B4FE43
:100D4400832584FE2320B4FE232204FE832504FE8F
:100D54009398050013080000232004FF232214FFA6
:100D64008325C4FE1387050093070000832504FE32
:100D740033E6E500832544FEB3E6F5002320C4FEF4
:100D84002322D4FE032704FE832744FE1305070011
:100D9400938507000324C101130101026780000049
:100DA400130101FF232611002324810013040101F0
:100DB400B72700001385C7AEEFF00FCAB7270000AE
:100DC4001385C7B0EFF04FC9B7270000138507B3E9
:100DD400EFF08FC8B7270000138587B5EFF0CFC7B2
:100DE400B72700001385C7B8EFF00FC71300000042
:100DF4008320C100032481001301010167800000E6
:100E0400130101E8232E1116232C8116232A2117FE
:100E1400232831172326411723245117232261172E
:100E240023207117130401182326A4E82324B4E80B
:100E3400B70700F0232CF4FCB70700F093870701F1
:100E4400232AF4FCB7C7010013850720EFF09FBAEB
:100E5400232804FC232604FCEFF01FE513090500F6
:100E640093890500EFF01FEC130705009387050035
:100E74001306400693060000130507009385070038
:100E8400EF00404113070500938705001306070090
:100E9400938607001305090093850900EF00803F3E
:100EA40013070500938705002324E4FCEFF0CFA883
:100EB40093070500638E0708EFF01FDF930704E92B
:100EC40013070003930680001386050093050500AD
:100ED40013850700EFF00FE2930704E91385070079
:100EE400EFF08FB7B7270000138547BAEFF0CFB6FE
:100EF400EFF05FE3930704E9130700039306800010
:100F0400138605009305050013850700EFF08FDEB7
:100F1400930704E913850700EFF00FB4B727000027
:100F2400138547BAEFF04FB3930704E9832584FC94
:100F340013850700EFF04FC6930704E913850700F4
:100F4400EFF08FB1B7270000138587BAEFF0CFB069
:100F5400EFF04FA293070500E38C07FE930704E923
:100F64009305F00F13850700EFF08FB51300000011
:100F7400B72700001385C7BAEFF00FAE930704E953
:100F840013850700EFF04FADB7270000138507BBAB
:100F9400EFF08FAC130704E913064000B7270000F5
:100FA400938547BB13050700EFF05F9B930705008C
:100FB40063960700EFF0DFDE6FF01FEA034704E9F2
:100FC40093072006631CF702930704E9938727001D
:100FD4009305000013850700EFF04FEC2326A4FAD5
:100FE4008327C4FA6358F0000325C4FAEFF09FA0E6
:100FF4006FF09FE6EFF0DFDA6FF01FE6034704E9D6
:1010040093074006631AF702930704E993872700BE
:101014009305000013850700EFF00FF82328A4FAC6
:10102400832704FB6356F000032704FB23ACE1C2CF
:10103400EFF05FA06FF05FE2034704E993077007E6
:10104400631CF70A930704E993872700130744F9FD
:101054009305070013850700EFF00FF4232EA4FA7D
:10106400832744F9130744F9930507001385070000
:10107400EFF08FF2232CA4FA832744F9130744F9E1
:101084009305070013850700EFF00FF1232AA4FA54
:10109400032744FB93071000631CF7008327C4FB5A
:1010A400032784FB1377F70F2380E7006FF0DFDA61
:1010B400032744FB93072000631EF7008327C4FB28
:1010C400032784FB13170701135707412390E700F5
:1010D4006FF09FD8032744FB93074000631AF7007F
:1010E4008327C4FB032784FB23A0E7006FF0DFD62C
:1010F400EFF01FCB6FF05FD6034704E99307200797
:10110400E31CF7D4232E04FC930704E993872700F8
:10111400130704F99305070013850700EFF0CFE7E1
:101124002322A4FC832704F9130704F99305070079
:1011340013850700EFF04FE62320A4FC032704FCEB
:10114400930710006310F702832744FC83C707004A
:10115400232EF4FCB72700001385C7BBEFF0CF8F15
:101164006F008005032704FC930720006310F70237
:10117400832744FC83970700232EF4FCB727000041
:10118400138547BCEFF04F8D6F000003032704FC69
:10119400930740006310F702832744FC83A70700EA
:1011A400232EF4FCB72700001385C7BCEFF0CF8AC9
:1011B4006F008000EFF0DFBE032704FC93071000EC
:1011C400630EF700032704FC930720006308F7006D
:1011D400032704FC93074000E310F7C8832744FC6B
:1011E400138A070093D7F741938A0700930704E90A
:1011F400130700039306800093050A0013860A0070
:1012040013850700EFF00FAF930704E91385070078
:10121400EFF08F84B7270000138547BDEFF0CF832D
:10122400930704E98325C4FD13850700EFF0CF96E7
:10123400930704E913850700EFF00F82B727000036
:10124400138587BDEFF04F818327C4FD138B0700FF
:1012540093D7F741938B0700832704FC93961700D9
:10126400930704E91307000393050B0013860B008F
:1012740013850700EFF00FA8930704E9138507000F
:10128400EFE09FFDB72700001385C7BDEFE0DFFC4B
:101294006FF09FBC13030500938805001307060035
:1012A400130805009387050063920628B7250000FC
:1012B400938505BE63F6C80EB70601006378D60CA5
:1012C4009336061093C61600939636003355D6000F
:1012D400B385A50083C5050013050002B386D500B8
:1012E400B305D540630CD500B397B800B356D3000B
:1012F4003317B600B3E7F6003318B300935507016C
:1013040033D3B7021316070113560601B3F7B70216
:1013140013050300B3086602939607019357080167
:10132400B3E7D70063FE1701B387E7001305F3FFA4
:1013340063E8E70063F617011305E3FFB387E700EB
:10134400B3871741B3D8B70213180801135808011B
:10135400B3F7B702B3061603939707013368F8008F
:1013640093870800637CD800330807019387F8FF4C
:101374006366E8006374D8009387E8FF13150501DA
:101384003365F50093050000678000003705000110
:1013940093060001E36CA6F2930680016FF01FF33D
:1013A4006314060073001000B70701006370F60CA5
:1013B4009336061093C6160093963600B357D6009C
:1013C400B385F50083C70500B387D70093060002F1
:1013D400B385F6406396F60AB387C84093051000B8
:1013E4009358070133DE170313160701135606013A
:1013F40093560801B3F7170313050E003303C6030E
:1014040093970701B3E7F60063FE6700B387E7002D
:101414001305FEFF63E8E70063F667001305EEFFBC
:10142400B387E700B387674033D317031318080162
:1014340013580801B3F71703B3066602939707011D
:101444003368F80093070300637CD800330807016E
:101454009307F3FF6366E8006374D8009307E3FF20
:10146400131505013365F50067800000B707000117
:1014740093060001E364F6F4930680016FF01FF411
:101484003317B600B3D6F80013550701B357F3006A
:101494003318B30033D3A60213160701B398B80068
:1014A40013560601B3E71701B3F6A602B3086602A2
:1014B4009395060193D60701B3E6B600930503009E
:1014C40063FE1601B386E6009305F3FF63E8E600C6
:1014D40063F616019305E3FFB386E600B38616416F
:1014E400B3D8A6029397070193D70701B3F6A602D0
:1014F4003306160393960601B3E7D70093860800D4
:1015040063FEC700B387E7009386F8FF63E8E7004C
:1015140063F6C7009386E8FFB387E7009395050158
:10152400B387C740B3E5D5006FF09FEB63E6D518EA
:10153400B707010063F4F60413B706101347170046
:1015440013173700B7270000B3D5E600938707BE0B
:10155400B387B70083C70700B387E7001307000208
:10156400B305F7406316F70213051000E3EE16E126
:101574003335C3001345150067800000B707000129
:1015840013070001E3E0F6FC130780016FF09FFBF3
:101594003357F600B396B600B366D70033D7F800D6
:1015A400B398B800B357F300B3E7170193D8060113
:1015B400B35E170313980601135808013316B600D7
:1015C40033771703330ED8031315070113D7070115
:1015D4003367A70013850E00637EC7013307D70066
:1015E4001385FEFF6368D7006376C7011385EEFF9A
:1015F4003307D7003307C741335E170393970701B7
:1016040093D70701337717033308C8031317070168
:10161400B3E7E70013070E0063FE0701B387D700A3
:101624001307FEFF63E8D70063F607011307EEFF15
:10163400B387D70013150501370E01003365E500A4
:101644009306FEFF3377D500B3870741B376D60000
:101654001358050113560601B308D702B306D8027E
:101664003307C7023308C8023306D70013D708016B
:101674003307C7006374D7003308C80193560701C2
:10168400B386060163E6D702E39ED7CEB70701000F
:101694009387F7FF3377F70013170701B3F8F800C0
:1016A4003313B3003307170193050000E37EE3CC43
:1016B4001305F5FF6FF01FCD93050000130500001F
:1016C40067800000130101FF9305000023248100BB
:1016D4002326110013040500EF00401903A581C25D
:1016E4008327C50363840700E7800700130504000C
:1016F400EF00403A130101FF23248100232021013C
:1017040037240000372900009307C4021309C902D3
:101714003309F9402326110023229100135929404B
:10172400630009021304C402930400008327040025
:101734009384140013044400E7800700E31899FE1F
:1017440037240000372900009307C4021309490312
:101754003309F94013592940630009021304C402F0
:1017640093040000832704009384140013044400AA
:10177400E7800700E31899FE8320C1000324810059
:101784008324410003290100130101016780000043
:101794001303F00013070500637EC3029377F70079
:1017A4006390070A63920508937606FF1376F600A2
:1017B400B386E6002320B7002322B7002324B70012
:1017C4002326B70013070701E366D7FE6314060058
:1017D40067800000B306C34093962600970200007A
:1017E400B38656006780C6002307B700A306B70078
:1017F4002306B700A305B7002305B700A304B70069
:101804002304B700A303B7002303B700A302B70060
:101814002302B700A301B7002301B700A300B70058
:101824002300B7006780000093F5F50F93968500B9
:10183400B3E5D50093960501B3E5D5006FF0DFF667
:101844009396270097020000B38656009382000007
:10185400E78006FA93800200938707FF3307F74077
:101864003306F600E378C3F66FF0DFF3130101FDEE
:10187400232C410103AA81C2232021032326110220
:1018840003298A142324810223229102232E310165
:10189400232A510123286101232671012324810174
:1018A40063000904130B0500938B0500930A1000D1
:1018B4009309F0FF832449001384F4FF6342040274
:1018C40093942400B304990063840B0483A7441005
:1018D400638077051304F4FF9384C4FFE31634FF95
:1018E4008320C102032481028324410203290102CB
:1018F4008329C101032A8101832A4101032B0101A8
:10190400832BC100032C81001301010367800000B5
:101914008327490083A644009387F7FF638E8704D7
:1019240023A20400E38806FA8327891833978A00E0
:10193400032C4900B377F70063920702E78006009F
:101944000327490083278A1463148701E38427F952
:10195400E38807F8138907006FF0DFF58327C918B8
:1019640083A544083377F700631C070013050B00B5
:10197400E78006006FF0DFFC232289006FF09FFAF6
:1019840013850500E78006006FF09FFB130101FF3C
:1019940023248100B72700003724000093874703DE
:1019A400130484033304F4402322910023261100FA
:1019B40093542440638004021304C4FF3304F400EA
:1019C400832704009384F4FF1304C4FFE780070013
:1019D400E39804FE8320C100032481008324410092
:1019E40013010101678000009305050093060000C0
:1019F40013060000130500006F00400003A781C216
:101A040083278714638C070403A747001308F00196
:101A1400634EE806131827006306050233830701A3
:101A24002324C30883A88718130610003316E6007E
:101A3400B3E8C80023A417192324D3109306200065
:101A44006304D5021307170023A2E700B387070135
:101A540023A4B70013050000678000009307C71490
:101A64002324F7146FF05FFA83A6C718130717002F
:101A740023A2E700B3E6C60023A6D718B38707015D
:101A840023A4B70013050000678000001305F0FFCE
:101A9400678000009308D0057300000063440500CC
:101AA4006F000000130101FF2324810013040500CB
:101AB4002326110033048040EF00C000232085005A
:0C1AC4006F00000003A501C36780000054
:101AD0002020000020202000200000002D200000F9
:101AE00020207C007C0A00000A00000020206420E6
:101AF0003C616464723E202D2D20646973706C61BA
:101B000079206D656D6F7279200A000020206220B7
:101B10003C62617564726174653E202D2D20736591
:101B200074206261756472617465200A00000000AF
:101B3000202072203C616464723E203C77696474AA
:101B4000683E202D2D2072656164206D656D6F7279
:101B50007920776F72640A00202077203C616464EA
:101B6000723E203C76616C75653E203C77696474FA
:101B7000683E202D2D207772697465206D656D6F2C
:101B8000727920776F72640A000000002020202004
:101B900077696474683D312C2032206F7220340ADA
:101BA000000000003A0000003E3E00000A0D3A002E
:101BB0000A0D000068656C702000000063686172A7
:101BC0002040000073686F7274204000696E7420BA
:101BD00040000000203D200028000000290A0D00E0
:101BE00000010202030303030404040404040404C4
:101BF0000505050505050505050505050505050595
:101C00000606060606060606060606060606060674
:101C10000606060606060606060606060606060664
:101C20000707070707070707070707070707070744
:101C30000707070707070707070707070707070734
:101C40000707070707070707070707070707070724
:101C50000707070707070707070707070707070714
:101C600008080808080808080808080808080808F4
:101C700008080808080808080808080808080808E4
:101C800008080808080808080808080808080808D4
:101C900008080808080808080808080808080808C4
:101CA00008080808080808080808080808080808B4
:101CB00008080808080808080808080808080808A4
:101CC0000808080808080808080808080808080894
:101CD0000808080808080808080808080808080884
:102000001000000000000000037A5200017C010172
:102010001B0D020010000000180000007CF2FFFF02
:0C20200030040000000000000000000080
:08202C00740000001C0100001B
:04203400D8000000D0
:1020380000000000242300008C230000F42300008B
:102048000000000000000000000000000000000088
:102058000000000000000000000000000000000078
:102068000000000000000000000000000000000068
:102078000000000000000000000000000000000058
:102088000000000000000000000000000000000048
:102098000000000000000000000000000000000038
:1020A8000000000000000000000000000000000028
:1020B8000000000000000000000000000000000018
:1020C8000000000000000000000000000000000008
:1020D80000000000000000000100000000000000F7
:1020E8000E33CDAB34126DE6ECDE05000B000000BC
:1020F80000000000000000000000000000000000D8
:1021080000000000000000000000000000000000C7
:1021180000000000000000000000000000000000B7
:1021280000000000000000000000000000000000A7
:0C24600038200000000100F038200000CF
:040000030000008C6D
:00000001FF
